:100000000C94AB010C94C8010C94C8010C94C80169
:100010000C94C8010C94C8010C94C8010C94C8013C
:100020000C94C8010C94C8010C9491220C94632385
:100030000C94831D0C94C8010C94C8010C94C80145
:100040000C94C8010C94C8010C94C8010C94C8010C
:100050000C94C8010C940B1E0C94C8010C94C8019C
:100060000C94C8010C94C8010C94C8010C94C801EC
:100070000C94C8010C94C8010C94C8010C94C801DC
:100080000C94C8010C94C8010C94C8010C94C801CC
:100090000C94C8010C94C8010C94C8010C94C801BC
:1000A0000C94C8010C94C8010C94C8014505450581
:1000B00071057105D905F7050F070F0702069B06A5
:1000C000AC06AC06D023F723EF24F723EF24432418
:1000D0006624EF24BD24CC24F400F200ED00F100EE
:1000E000F500EF00EE00F000FD00FE00FF00000054
:1000F00000010101010101010101020202020202EB
:1001000002020203030303030303030404040404BD
:100110000404050505050506060606060707070784
:100120000708080808090909090A0A0A0B0B0B0C39
:100130000C0C0D0D0D0E0E0E0F0F0F1010111111D6
:100140001212131314141515161617171818191957
:100150001A1A1B1B1C1D1D1E1E1F202021222223BC
:100160002424252626272829292A2B2C2D2D2E2FFD
:1001700030313232333435363738393A3B3C3D3E14
:100180003F404142434445464748494A4C4D4E4F03
:1001900050515354555658595A5B5D5E5F616264C5
:1001A000656668696B6C6D6F7072737577787A7B52
:1001B0007D7E8082838587888A8C8E8F91939596A9
:1001C000989A9C9EA0A2A3A5A7A9ABADAFB1B3B5C9
:1001D000B7BABCBEC0C2C4C6C9CBCDCFD1D4D6D8A5
:1001E000DBDDDFE2E4E7E9EBEEF0F3F5F8FAFDFF43
:1001F00010034C0079006E0065007000610064001F
:1002000000000A0351005600450058000000040396
:10021000090409023B00020100A0FA0904000001E0
:10022000030101000921110100012240000705819D
:100230000308000109040100010300000009211165
:1002400001000122B600070582032000011201000F
:1002500002000000085651504C0100010200010547
:10026000010902A10185020901A10005091901295D
:10027000081500250195087501810205010930095D
:10028000311581257F95027508810609381581256C
:100290007F950175088106050C0A38021581257FB6
:1002A000950175088106C0C005010980A10185037B
:1002B00019012AB700150126B700950175108100B4
:1002C000C0050C0901A101850419012AA00215012C
:1002D00026A002950175108100C005010906A10143
:1002E0008506050719E029E7150025019508750120
:1002F00081020507190029EF1500250195F0750108
:1003000081020508190129059505750191029501DC
:1003100075039101C005010906A101050719E0292E
:10032000E715002501950875018102950175088181
:10033000010507190029FF150026FF00950675081D
:10034000810005081901290595057501910295019E
:1003500075039101C00011241FBECFEFDAE0DEBFAC
:10036000CDBF11E0A0E0B1E0E0E5FBE402C0059004
:100370000D92A63BB107D9F722E0A6EBB1E001C090
:100380001D92AC3CB207E1F70E9408130C94A6251D
:100390000C94000052985A983E98469854985C984D
:1003A00026982E9857985F9824982C980C94CE0EE7
:1003B000809116019091170190931501809314017B
:1003C00089B182FB882780F980931601109217016A
:1003D000809112019091130190931101809310016B
:1003E00086B186FB882780F9809312011092130151
:1003F00080910E0190910F0190930D0180930C015B
:1004000089B18295817080930E0110920F018091C5
:100410000A0190910B01909309018093080183B127
:1004200086FB882780F980930A0110920B01809146
:10043000060190910701909305018093040189B111
:10044000082E000C990B892F881F8827881F8093FE
:10045000060110920701809102019091030190938F
:1004600001018093000183B1829581708093020124
:10047000109203010C944F02811106C0662311F003
:100480008AEA09C089EA07C0813039F4662311F08D
:1004900089EF01C08AEF0E94F30481E00895809102
:1004A00016019091170120911401309115018217C6
:1004B000930729F01816190614F40E946F0380910F
:1004C00012019091130120911001309111018217B6
:1004D000930759F01816190624F083EF90E00C9456
:1004E000EC0283EF90E00C94020380910E01909156
:1004F0000F0120910C0130910D018217930729F013
:100500001816190614F40E949E1780910A01909102
:100510000B0120910801309109018217930729F0FE
:100520001816190614F40E94B017809106019091D4
:10053000070120910401309105018217930729F0EA
:100540001816190614F40E943B188091020190912C
:10055000030120910001309101018217930729F0D6
:100560001816190614F40C94DA1708959C013A959C
:1005700021153F4130F5BC0166277270AC0144275C
:1005800054709C012227387094FF0FC090FF02C066
:1005900080E101C080E0672B09F08062452B09F003
:1005A0008064232B79F080680895892F8170672BF0
:1005B00009F08260452B09F08460232B19F08860D4
:1005C000089580E00895CF93DF93EB010E94B60277
:1005D000FE01DF91CF910994CF93DF93EC01805E10
:1005E0009109089710F0209719F46CEF74E002C09D
:1005F00067E877E0CE010E94E3028C2FDF91CF9174
:100600000C945204CF93DF93EC010E94A804CE0116
:10061000805E9109089710F0209719F463E075E067
:1006200002C06EE877E0CE01DF91CF910C94E30237
:1006300081E0089581E008950C941A0308950C94C4
:100640001E031F93CF93DF9300D000D01F92CDB72E
:10065000DEB749835A836B833091B90189819A81CE
:10066000311114C0662359F0222349F00E94580921
:10067000182F682F89819A810E94030903C00E9464
:100680002D09182F69817A81812F04C00E94580991
:1006900069817A810F900F900F900F900F90DF91EA
:1006A000CF911F910C949310FC01262F4081518112
:1006B0006281738184810C94210381E00895CF933A
:1006C000DF93EC0160E00E945403BE01DF91CF9103
:1006D0000C941F030C94D7110C94D80108950E9418
:1006E000AD070E946E032FEF84E39CE02150804011
:1006F0009040E1F700C000000C94311E0F931F934F
:10070000CF93DF938C0161E00E945403EC01B801A8
:100710000E941C03882309F444C0B801CE010E9442
:10072000CF1B8823F1F1B801CE010E94EA1888237B
:10073000C1F1B801CE010E942B1B882391F1B801B1
:10074000CE010E944818882361F1F8018281882334
:1007500009F1CB358DE5D807C1F050F4C115FCE5A2
:10076000DF0781F0CF3DDC45A9F40E948F0E19C050
:10077000CC35EDE5DE0761F0CD35DD4559F40E945D
:10078000D20D08C00E946F030CC00E94DB0D02C096
:100790000E94DE0DC801DF91CF911F910F910C9443
:1007A000180380E0DF91CF911F910F9108950E946F
:1007B000661D0C94F0030E94F3030C946C1D0895C5
:1007C0000C94DF0381E008950C94E2030895CF9325
:1007D000C82F0E94E0038C2F0E94E403CF9108955C
:1007E00080E00C94E7030E942B1C0C94E7030E940A
:1007F0002B1C9091B801891721F08093B8010C94BB
:10080000E7030895CF93DF93CDB7DEB72B970FB6ED
:10081000F894DEBF0FBECDBF4F83588769877A87B4
:100820008B8761110E941E0D9E012F5F3F4F86E056
:10083000F90111928A95E9F785E0FE013796D90111
:1008400001900D928A95E1F789819A814C815D81B1
:10085000452B31F09F3F31F491E08F3F19F403C0F5
:1008600091E001C090E090FF09C049815A816B81FD
:100870007C818D819E810E943F0C05C0C9010E9430
:100880005D038111F2CF2B960FB6F894DEBF0FBE39
:10089000CDBFDF91CF910895FC01808191810E94AD
:1008A0009A090895CF93882309F450C0C82F8CEF7C
:1008B0008C0F813AD0F46C2F80911A0190911B011A
:1008C0000E94A11C882349F06C2F80911A019091FD
:1008D0001B010E942C1D0E94400D6C2F80911A015B
:1008E00090911B010E94211D0CC080E28C0F88306A
:1008F00058F4C77081E001C0880FCA95EAF70E94DA
:10090000010DCF910C94400DEBE5EC0FE33040F47A
:10091000F0E0EC59FE4F808190E0CF910C945F1C89
:10092000E8E5EC0FE73150F4F0E0EE0FFF1FEA5C72
:10093000FE4F80819181CF910C94751CCD3E30F09B
:100940008C2F0E948D13CF910C945F14CF9108953A
:10095000882389F19CEF980F913A40F4682F809199
:100960001A0190911B010E942C1D0DC090E2980F5E
:10097000983058F4877091E001C0990F8A95EAF792
:10098000892F0E94070D0C94400D9BE5980F933022
:1009900020F480E090E00C945F1C98E5980F97316C
:1009A00020F480E090E00C94751C8D3E20F00E94B5
:1009B000E8130C945F1408951F93CF93DF93182FBF
:1009C000EB010E945204209741F08FE99FE00197CC
:1009D000F1F700C000002197F6CF812FDF91CF9172
:1009E0001F910C94A804893319F060E070E002C0F4
:1009F00060E570E00C94DC04882321F00E94010D76
:100A00000C94400D0895882321F00E94070D0C944A
:100A1000400D0895CF92DF92EF92FF920F931F93B4
:100A2000CF93DF937C01D62FC72FFC011281058164
:100A300002950F700E94F70C8823B9F01123A9F0DA
:100A40008C2F807F803421F080E28D0F883068F019
:100A50008091A30282FD09C082E00E94A00D0E9445
:100A6000F70C91E0D82ED92601C0D12CCC2EC294FF
:100A70008FE0C8228C2D90E08C30910508F0CFC11A
:100A8000FC01EA5AFF4F0C944B258C2F807FCF70CE
:100A9000882311F0C295C07F112399F0CC2309F46B
:100AA000AAC180E28D0F883010F0D11104C08C2FC4
:100AB0000E94010D03C08C2F0E94110D0E94400D59
:100AC0009AC18D2F0E94A804CC2309F4A8C180E20A
:100AD0008D0F883038F1DD2329F18C2F0E94170DFE
:100AE00024C08C2F807FCF70803211F0C295C07FE0
:100AF000DD2319F0D130A1F13DC08091A30282FF26
:100B000017C0112349F0CC2329F08C2F0E94010D2E
:100B10000E94400D80E070C180E00E94A804CC23B8
:100B200009F47DC18C2F0E94070D0E94400D77C1F2
:100B3000112371F0002341F0013031F40E94210DA6
:100B40008C2B0E94290D6BC10E94210D8C2B1DC086
:100B5000002319F0013009F462C10E94360D25C04E
:100B6000112321F0063008F05AC10EC0053008F0FC
:100B700056C11BC0112361F0002331F0F7018581BC
:100B800080FF39C18F7085838C2F0E94FC0447C180
:100B9000002359F0D93309F03FC1FFEF07EE13E00E
:100BA000F15000401040E1F735C18C2F0E94030541
:100BB00036C18C2F86958695837019F0813061F04F
:100BC0002EC1112321F08D2F9C2F937002C080E045
:100BD00090E00E945F1C2BC1112321F08D2F9C2FD0
:100BE000937002C080E090E00E94751C20C18D2FA0
:100BF000112319F00E948D1302C00E94E8130E9475
:100C00005F1415C18C2F837009F047C011110BC1FF
:100C10002D2F229526952770220F220F6D2F6F7092
:100C2000862F90E0A0E0B0E0022E04C0880F991F4C
:100C3000AA1FBB1F0A94D2F7D4FF10C04FE050E0A8
:100C400060E070E004C0440F551F661F771F2A95AF
:100C5000D2F7409550956095709503C040E050E004
:100C6000BA01C695C695C3708A019B01082B192B42
:100C70002A2B3B2BC901B801C23049F058F4C130CE
:100C800019F00E941908CFC00E940708CCC00E942A
:100C90002B08C9C00E940508C6C0112319F08C2F6B
:100CA000817001C08695882309F4BDC02D2F22953F
:100CB00026952770220F220F6D2F6F70862F90E0E0
:100CC000A0E0B0E0022E04C0880F991FAA1FBB1F2E
:100CD0000A94D2F7D4FF10C04FE050E060E070E01B
:100CE00004C0440F551F661F771F2A95D2F7409501
:100CF00050956095709503C040E050E0BA01C695EC
:100D0000C695C3708A019B01082B192B2A2B3B2BFC
:100D1000C901B801C23049F058F4C13019F00E943D
:100D2000DE0881C00E94CC087EC00E94F0087BC013
:100D30000E943F0878C0CF70112339F08C2F0E9499
:100D400065088D2F0E94FC046EC08D2F0E94030544
:100D50008C2F0E94860867C0D23F21F128F4D03F33
:100D600041F0D13FC1F043C0D33F19F1D43F79F0F6
:100D70003EC0112341F0053008F051C08C2F8F7117
:100D80000E94AB084CC0063008F049C0F7CF8091F4
:100D9000A30282FF18C0112339F08C2F8F710E949B
:100DA00065083DC01123C9F38C2F8F710E948608FE
:100DB00036C0112329F08C2F8F710E9450082FC04C
:100DC0000E944B082CC0112349F0CF718C2F0E9438
:100DD000650863E08C2F0E94850D21C081E00E9490
:100DE000A00D0230E0F082E00E94A00D18C0112397
:100DF00031F0002391F28D2F0E94520410C0002385
:100E000099F2D93349F41FEF27EE33E01150204017
:100E10003040E1F700C000008D2F0E94A80488EF49
:100E20008C0D843020F40E942B1C0E94E703DD20EF
:100E3000C9F00E94F30C80FD15C0F70112820E94D8
:100E4000ED0C0E946508C7010E9453070E94ED0C3B
:100E5000DF91CF911F910F91FF90EF90DF90CF9096
:100E60000C948608DF91CF911F910F91FF90EF9026
:100E7000DF90CF9008950F931F93CF93DF93EC01F2
:100E8000688179818A810E94A5098C010E940209EA
:100E90000E94F307B801CE010E940A05DF91CF91AD
:100EA0001F910F910895CF93DF93EC019881898171
:100EB0002B813C81232B31F08F3F31F481E09F3F28
:100EC00019F403C081E001C080E080FD1DC0CE01A7
:100ED0000E947E03811110C00E94F70C8823A1F0AC
:100EE0008A81882389F08091A30282FD0DC082E06F
:100EF000DF91CF910C94A00DCE010E943B07CE0153
:100F0000DF91CF910C945F03DF91CF9108958823F7
:100F100021F00E94110D0C94400D0895882321F0BA
:100F20000E94170D0C94400D089580E090E00E94FF
:100F30005F1C80E090E00E94751C0E941E0D0E94C4
:100F4000400D0E9490150C945F1480911A019091AD
:100F50001B010E94371D0C9495070E940E0D0C94E6
:100F6000A50792959F70963079F010F4925001C0C9
:100F70009A50923068F4803F69F018F4883E40F44B
:100F800009C0843F29F406C0883E20F0813F11F05B
:100F900080E0089581E00895FC01808191810E94A4
:100FA0009A090E94B1070895CF93DF9300D000D033
:100FB0001F92CDB7DEB70F900F900F900F900F904C
:100FC000DF91CF910895CF93DF9300D000D000D070
:100FD000CDB7DEB726960FB6F894DEBF0FBECDBFF5
:100FE000DF91CF910895089508950C94F4070C941F
:100FF000F5070E94F7076093C8017093C9018093B9
:10100000CA019093CB010C9495070C94F9070F93A8
:101010001F930091C8011091C9012091CA0130911C
:10102000CB01602B712B822B932B1F910F910C9472
:10103000F9070F931F930091C8011091C9012091E6
:10104000CA013091CB0160237123822393231F9126
:101050000F910C94F9070F931F930091C801109101
:10106000C9012091CA013091CB01602771278227E5
:1010700093271F910F910C94F9070C94F4070E9489
:101080003D086093C4017093C5018093C60190939D
:10109000C7010C94950760E070E0CB010C943F0809
:1010A0000F931F9341E050E060E070E08A019B01E4
:1010B00004C0000F111F221F331F8A95D2F7C901E8
:1010C000B8011F910F910C943F080F931F9341E0BB
:1010D00050E060E070E004C0440F551F661F771FAA
:1010E0008A95D2F78091C4019091C501A091C60163
:1010F000B091C7018A019B01082B192B2A2B3B2B8E
:10110000C901B8011F910F910C943F080F931F93D1
:1011100041E050E060E070E004C0440F551F661FDE
:10112000771F8A95D2F7409550956095709580917C
:10113000C4019091C501A091C601B091C7018A0177
:101140009B01082319232A233B23C901B8011F91BE
:101150000F910C943F080F931F9341E050E060E023
:1011600070E004C0440F551F661F771F8A95D2F7A1
:101170008091C4019091C501A091C601B091C701B1
:101180008A019B01082719272A273B27C901B80193
:101190001F910F910C943F080F931F930091C4016E
:1011A0001091C5012091C6013091C701602B712BB0
:1011B000822B932B1F910F910C943F080F931F9339
:1011C0000091C4011091C5012091C6013091C70161
:1011D00060237123822393231F910F910C943F0866
:1011E0000F931F930091C4011091C5012091C60176
:1011F0003091C70160277127822793271F910F9194
:101200000C943F080895990F990F890FE82FE695E0
:10121000E695E695877051E001C0550F8A95EAF78B
:1012200085E0E89FF0011124E654FE4F20E030E015
:1012300070E04081CB01022E02C0969587950A94FA
:10124000E2F78170819584278523842781932F5F1E
:101250003F4F2530310569F70895990F990F890F90
:10126000682F669566956695982F977085E0689FBC
:10127000B001112440E050E080E0FB01E40FF51FD5
:10128000E654FE4F208130E0092E02C036952795A6
:101290000A94E2F721703327042E01C0220F0A942A
:1012A000EAF7822B4F5F5F4F4530510531F70895C4
:1012B000BF92CF92DF92EF92FF920F931F93CF9343
:1012C000DF938C01C090C401D090C501E090C601AD
:1012D000F090C7018091C8019091C901A091CA0105
:1012E000B091CB01C82AD92AEA2AFB2ACFE1D0E063
:1012F000D701C6010C2E04C0B695A7959795879582
:101300000A94D2F780FD04C0219790F7B12C07C052
:10131000BC2EB8018C2F0E94A8100197A9F38B2D29
:10132000DF91CF911F910F91FF90EF90DF90CF90C1
:10133000BF900895CF93DF93EC010E945809BE013E
:101340000E94A810DF91CF9108951F93CF93DF9350
:10135000EB019091B901992321F0CB010E949A09E8
:1013600013C0882349F0CB010E945809182F682F19
:10137000CE010E94030904C0CB010E942D09182F41
:10138000BE01812F0E94A810DF91CF911F91089577
:101390001F93CF93DF93C091CC0116E08091CD01D4
:1013A000C81799F0D0E01C9FF0011D9FF00D11248B
:1013B000E253FE4F40815181628173818481958126
:1013C0000E94E3072196C770E9CFDF91CF911F916B
:1013D00008954091FE015091FF01609100027091CB
:1013E000010280910202909103020C94E307EF92B4
:1013F000FF920F931F93CF93DF9380910302829507
:101400008F7009F065C080910002882309F460C0E4
:101410008091CC01F090CD011091FE010091FF016F
:10142000609101027091020291E01F3F09F090E08B
:10143000C0911801D0911901292F96E0E92E8F153E
:1014400009F446C06115710521F00F3F21F030E02D
:1014500003C031E001C0322F90E030FD36C0E89E7D
:10146000F001E99EF00D1124DF01A253BE4F119649
:101470003C911197301329C03C91311326C012962C
:101480003C911297311121C013964D915C911497A4
:10149000461B570B4C175D07C0F4809103028F70F9
:1014A000806180930302ED52FE4F80818F708061D6
:1014B00080838EEF91E00E945307DF91CF911F91BF
:1014C0000F91FF90EF900C94C80901968770B7CFE9
:1014D000DF91CF911F910F91FF90EF9008959F9210
:1014E000AF92BF92CF92DF92EF92FF920F931F9332
:1014F000CF93DF93CDB7DEB761970FB6F894DEBF19
:101500000FBECDBF8C0185E0F801DE011D96019074
:101510000D928A95E1F7D8011296EC909091FE0118
:10152000E091FF0120910102309102022115310565
:1015300031F0EF3F31F481E09F3F19F403C081E0C7
:1015400001C080E0B82FB1709B2E80FD47C1D8014B
:101550004C9111965C9111971396AD90BC90149795
:101560008EEFC82E81E0D82EF0900002B501621BEC
:10157000730B2091180130911901FF2009F4D9C093
:10158000809103026217730708F095C0282F207F0F
:1015900009F052C05E1313C0491311C0FE2CE110B4
:1015A0000EC08F708061809303020E94E909C6011A
:1015B0000E94530780910302F80185834DC1AB2837
:1015C00031F05F3F31F481E04F3F19F403C081E017
:1015D00001C080E080FD03C081E08E2502C080E074
:1015E00090E0F82FF170FF2E80FF1CC08091CC019D
:1015F0002091CD0136E0821709F40BC190E0389FAD
:10160000F001399FF00D1124E253FE4F6181561312
:1016100006C06081461303C06281E61203C00196D2
:101620008770E9CFFE2CEE2009F416C180910302E9
:1016300081608093030254C05E1306C0491304C046
:10164000E11002C0F80199C0C8010E94CC078823AC
:1016500061F1EE2051F120910302822F82958F706B
:1016600090E0029774F08091FE019091FF019887BD
:101670008F831986BB86AA862C87CE0107960E9487
:10168000530786E0F801AEEFB1E001900D928A9524
:10169000E1F70E94F7090E94E9090AC05E1711F1FB
:1016A000C8010E94CC0781112CC0C8010E945307B9
:1016B000FF24F394D1C0282F207F81F77A2DB98A97
:1016C000A88A6E2D89890E94D4078EEF91E00E942E
:1016D000530786E0D6011D928A95E9F70E94E90931
:1016E000F12CBAC04913DCCFE110DACFF8018583C1
:1016F000C8010E94530786E0D6011D928A95E9F73A
:10170000ABC0EE2091F220910302822F82958F7060
:1017100090E002970CF4B5CF8091FE019091FF010B
:101720009A8389831B82BD82AC822E83CE0101966F
:10173000A6CF6217730708F044C0FE2CEE2009F410
:10174000B4CF5E1330C049132EC02091030220FD98
:1017500021C0822F82958F70482F50E0411551058E
:10176000C9F0F80125834F30510541F08F5F982F64
:101770009295907F822F8F70892B8583C8010E945C
:10178000530786E0F801AEEFB1E001900D928A9523
:10179000E1F73CC086E0F801AEEFB1E001900D92B8
:1017A0008A95E1F759C0C8010E94CC07811169CF21
:1017B00080910302816080930302C8010E94530755
:1017C0004BC07A2DB98AA88A6E2D89890E94D407C8
:1017D00086E0D6011D928A95E9F718C0EE2009F43B
:1017E00064CFC8010E94CC07F82E882309F45DCF8E
:1017F00086E0F801AEEFB1E001900D928A95E1F735
:101800008EEF91E00E944C040E94F7090E94E909C2
:1018100023C04D875E878D859E850E949A09292F5A
:1018200022952F70223028F49F7039F0811105C065
:101830000BC0243028F49F7049F4805E883020F07B
:10184000C8010E9453079F2CF92C06C0D801159699
:101850009C91907F91F7F8CF8F2D61960FB6F894F9
:10186000DEBF0FBECDBFDF91CF911F910F91FF90D3
:10187000EF90DF90CF90BF90AF909F9008951F930F
:10188000CF93DF93CDB7DEB72C970FB6F894DEBFBA
:101890000FBECDBF4F83588769877A878B879C8718
:1018A000CE0107960E946F0A8823D1F09F81888518
:1018B0002A853B85232B31F08F3F31F481E09F3F18
:1018C00019F403C081E001C080E080FD47C04F8172
:1018D000588569857A858B859C850E94E3073EC083
:1018E00086E0FE013796DE01119601900D928A95F1
:1018F000E1F7FF81E8856A857B856115710531F027
:10190000EF3F31F481E0FF3F19F403C081E001C0F3
:1019100080E080FD23C02091CD0130E0C901019617
:10192000877099274091CC0150E084179507F1F119
:10193000F983EA837D836C8396E0929FD001939F25
:10194000B00D1124A253BE4FFE01319601900D92AD
:101950009A95E1F78093CD010E94C80916E0809125
:10196000CC019091CD01891771F1189FC00111240C
:1019700082539E4F0E946F0A882329F1E091CC0187
:101980001E9FF0011124E253FE4F4081518162817C
:101990007381848195810E94E3078091CC0190E05E
:1019A0000196877099278093CC01D9CF0E94AD070B
:1019B0001092CD011092CC01EEEFF1E086E0DF0154
:1019C0001D928A95E9F72C960FB6F894DEBF0FBEEC
:1019D000CDBFDF91CF911F9108958091240285950D
:1019E000859585950895809124028770089590913A
:1019F0002402977081E009F480E008958091470205
:101A0000089590914702892B80934702089580950D
:101A100090914702892380934702089510924702CC
:101A2000089590914602892B8093460208958095EF
:101A300090914602892380934602089510924602AF
:101A4000089580912502089508950C94240D0C9416
:101A5000250D9091A30292FD08C090912502981740
:101A600021F0809325020C94270D08958091250282
:101A7000882329F01092250280E00C94270D089508
:101A8000CF93DF93E0911A01F0911B0180914702FF
:101A90008083E0911A01F0911B01908180914602B0
:101AA000892B808380912502882381F0E0911A019F
:101AB000F0911B019081892B808380911A01909174
:101AC0001B010E948B1C81110E94360DC0911A01CE
:101AD000D0911B0140E250E064E072E0CE010E9430
:101AE0005125892B69F080E2FE01A4E0B2E001906B
:101AF0000D928A95E1F7CE01DF91CF910C94371CBE
:101B0000DF91CF9108950C94240D9091A30292FD42
:101B100010C098E0899F90011124262B2093240265
:101B20000E946508809124028595859585950C9481
:101B3000830D0C9465081092240280E00C94830DB0
:101B4000209124028095822380932402982F9770FD
:101B500099F430E0482F082E000C550B2417350758
:101B600059F09091A30292FD07C0859585958595C2
:101B70000E9486080C949B0D08959091A30292FBFD
:101B8000222720F9281769F080FB92F99093A3028D
:101B90008091A2029091A3020E940B0E82E00C940D
:101BA000A00D08958091A30282FB882780F991E01F
:101BB00089270C94BD0D81E00C94BD0D80E00C9440
:101BC000BD0D6FEF7FEF80E090E00C94902580E0FA
:101BD00090E00E946C2521E0893E9E4F09F020E0B4
:101BE000822F089582E090E00C945E2583E090E0DF
:101BF0000C945E25CF9384E090E00E945E25C82F70
:101C000082E290E00E945E252C2F30E0A901582B43
:101C1000CA01CF910895CF93C92F682F84E090E037
:101C20000E9472256C2F82E290E0CF910C94722575
:101C3000AB01BC018FE090E00C948425AB01BC01AA
:101C400083E190E00C94842560E070E0CB010C947B
:101C50001E0E60E070E0CB010E94180E0C94240E62
:101C600069EE7EEF80E090E00E94902560E082E0E7
:101C700090E00E94722560E083E090E00E9472256F
:101C80001092C8011092C9011092CA011092CB01A2
:101C900060E084E090E00E94722560E082E290E0E3
:101CA0000E94722560E085E090E00E94722560E06D
:101CB00086E090E00E9472256FEF87E090E00E943E
:101CC000722540E050E0BA0188E090E00E9484254F
:101CD00060E08DE090E00E94722540E050E0BA01A3
:101CE00088E190E00E94842560E087E190E00E9416
:101CF000722540E050E0BA018CE190E00E9484251A
:101D000060E070E080E290E00E94902540E050E0CA
:101D1000BA0188E190E00E9484250C94290E0C946D
:101D2000300E682F8EE090E00C9472250E94F01D1A
:101D3000609353027093540280935502909356021D
:101D400060934F027093500280935102909352021D
:101D500008950E94F01D6093530270935402809383
:101D600055029093560260934B0270934C028093FD
:101D70004D0290934E02089585B7806885BF85B760
:101D8000806885BF089581E008950C94C30E08957E
:101D90000C94C70E0C94C70E0C94CA0E0C94C70E6C
:101DA0000C94C70E0E94BC0E84E891E10E94211C95
:101DB0000E94D00E0C94CA010E94C80E0C94C70E4B
:101DC0000E94A1110C94E6030E94DB1D0E946D127B
:101DD0000E94E00E0E9402180E943B1A0C94CC0E46
:101DE0008F929F92AF92BF92CF92DF92EF92FF922B
:101DF0000F931F93CF93DF93CDB7DEB72A970FB61C
:101E0000F894DEBF0FBECDBF0E948212982E8111C2
:101E10000E94960E88E4A82E82E0B82E00E010E022
:101E2000802E802F0E94C511D82EF501C1905F0130
:101E3000C826B1F40F5F1F4F0330110589F78FEFEC
:101E400089838A831B820E94E41D8160782F9D8391
:101E50008C8349815A816B818D810E9402042FC03D
:101E60008091570281FD0E94CB11E12CFF24F39455
:101E70008C2D8F21F1F00E94C50E882399F0EE82FF
:101E80008F82DF2081E009F480E088870E94E41DD2
:101E90008160782F9A8789874E815F8168858A85DE
:101EA0000E940204F801E85BFD4F8081F826F08271
:101EB00006C0E394FF0CF4E0EF12DACFBBCF81E071
:101EC000911001C080E02A960FB6F894DEBF0FBED5
:101ED000CDBFDF91CF911F910F91FF90EF90DF90D9
:101EE000CF90BF90AF909F908F9008950E94F00E7A
:101EF0000E948E1A81110E94A90E0E947D140C94DA
:101F0000F703CF93DF930E94AD10EC01811521E51B
:101F1000920708F045C0811530E5930708F094C09A
:101F2000883E910528F5803E910508F0F8C0883A72
:101F3000910570F4853A910508F07CC081309105D7
:101F400009F475C008F4E8C0049708F0E8C0E4C0DC
:101F50008F3B910508F0E0C0C85AD0E0CC0FDD1FE0
:101F6000C959DE4F0990D881C02DCE019464D8C0E4
:101F7000811540E2940758F4811551E0950708F067
:101F8000CEC08D3E910508F4C7C09065C9C0C1158B
:101F900080E4D80708F4C0C0DF70CE01906AC0C0EA
:101FA000811525E59207A8F4811534E5930708F01B
:101FB00095C0811543E5940708F07BC0811552E573
:101FC000950708F061C0D82FCC27CE01816F906AA9
:101FD000A7C0C11589E5D807A0F4C11528E5D20727
:101FE00008F082C0C11536E5D30708F095C08C2FE4
:101FF0000E9441118F7190E0D82FCC27CE019062C2
:102000008FC0C1154AE5D40708F474C0CE019056BC
:102010008115904208F080C08D2F8F710E94411170
:10202000DD27D0628F71AE01582BCA0179C081E0E3
:1020300090E076C0C55AD0E0CB56DE4F8881C82FDD
:10204000D0E0CE0190646CC074E0969587957A9547
:10205000E1F7282F23703C2F337081E090E002C01D
:10206000880F991F3A95E2F79C68AC01522B9A01B0
:102070009C2F9F709695969550E2959FE0011124B4
:10208000C9018C2B9D2B4CC08370992721E030E037
:1020900002C0220F331F8A95E2F79C2F96959695E2
:1020A00080E2989FE0011124C22BD32BCE019C68C3
:1020B00037C08370992721E030E002C0220F331F20
:1020C0008A95E2F79C2F9695969540E2949FE001C1
:1020D0001124C22BD32BCE019A6822C0D82FCC2733
:1020E000CE01846F906A1CC0DC2FCC27CE01806F9C
:1020F000906A16C08C2F8F700E94411194E0D69583
:10210000C7959A95E1F7CF70D0E0DC2FCC27D06946
:102110009E01282BC90104C080E090E001C0CE01DF
:10212000DF91CF91089590E0FC01EE0FFF1FE80FC3
:10213000F91FE70FF11DEE0FFF1FEE0FFF1FE60F58
:10214000F11DEE0FFF1FE852FF4F85919491089506
:102150000E9493100E94810F08958238910569F1C1
:10216000B0F48133910509F46DC048F489329105CA
:1021700009F463C08A32910509F469C00895853372
:10218000910509F455C089339105B9F00895833E4E
:10219000910569F138F4803E9105B1F0823E9105D8
:1021A00009F10895863E9105A9F1873E9105B9F19F
:1021B000843E910509F064C023C02091A20220FD55
:1021C0004FC021FD4DC008958091A20280FD44C002
:1021D0008091A30280FF44C08091A20284FD42C08E
:1021E00083EE4DC08091A20282FF38C0F5CF80916E
:1021F000A20282FD33C08091A30280FD31C0ECCFEA
:102200008091A30281FF32C08091A20284FD2AC086
:1022100087EE35C08091A20283FF26C0F5CF809162
:10222000A20283FD21C08091A30281FD1FC0ECCFDB
:102230008091A20285FD1CC01DC08091A20285FD77
:1022400019C016C08091A20286FD16C017C08091E9
:10225000A20286FD13C010C089E311C082EE0FC038
:1022600080EE0DC080E00BC086EE09C084EE07C092
:1022700089E205C085E303C08AE201C081E390E002
:1022800008959091A20292FF0DC0282F2871283046
:1022900019F4877F846006C0282F2471243011F43C
:1022A0008B7F886093FF0DC0282F2871283119F487
:1022B000877E846106C0282F2471243111F48B7E1F
:1022C00088612091A30220FF0DC0382F387138306B
:1022D00019F4877F816006C0382F3171313011F4D5
:1022E0008E7F886021FF0DC0282F2871283119F4B6
:1022F000877E816106C0282F2171213111F48E7EE5
:10230000886194FD877E089580E008950C94E10D26
:102310000E9482122FEF86E791E02150804090408A
:10232000E1F700C000000E94821280E00E94C51107
:1023300080FF04C00E9486110C94311E08950C94F5
:1023400088110E94E70D811102C00E948F0E0E9429
:10235000F20D809357020E94FA0D9093A30280938E
:10236000A2020E949F110E94F60D682F70E080E08B
:1023700090E00E9405086091C4017091C5018091B0
:10238000C6019091C7010C943D08E82FF0E0E95593
:10239000FD4F80810895089580EA8A95F1F70895A8
:1023A00000C008950C94CC1108950C94D4110C9491
:1023B000D511F894E82FE295EF70F0E031A1282FC5
:1023C0002F7081E090E001C0880F2A95EAF7982FDE
:1023D0009095932391A392A1892B82A37894089539
:1023E000CF93DF9387E60E94D91187EF0E94D9111E
:1023F00086EF0E94D911C8E9D1E089918F3F11F091
:102400000E94D91181E0CC39D807B9F7DF91CF917B
:102410000895CF92DF92EF92FF920F931F93CF9385
:10242000DF938C01C62FD0E0CE0184569E4F7C01F5
:10243000FC0190819F3F09F447C0D62EF894E92F04
:10244000E295EF70F0E081A19F7021E030E001C0E3
:10245000220F9A95EAF7822B81A382A12095282347
:1024600022A378940E94D011E8E9F1E04CE951E010
:1024700031E0C12C21912F3F89F0A22FA295AF709E
:10248000B0E090968C9190E02F7002C09595879562
:102490002A95E2F780FD02C0832F01C080E0C82AA0
:1024A000330F4E175F0731F7F70180818F3F11F02F
:1024B0000E94D91161E0C11001C060E08D2D0E9421
:1024C000D211C00FD11FC882DF91CF911F910F9100
:1024D000FF90EF90DF90CF9008950E94F01183E07D
:1024E000E7EAF2E0DF01982F1D929A95E9F7E4EA16
:1024F000F2E0DF011D928A95E9F783E00E94C512A0
:102500000C946A031F93CF93DF9300D01F92CDB733
:10251000DEB719821A821B8260E0CE0101960E940A
:10252000091261E0CE0101960E94091262E0CE011B
:1025300001960E94091243E050E0BE016F5F7F4F99
:1025400084EA92E00E94512511E0009709F410E01E
:10255000892B49F089819A81AB818093A402909361
:10256000A502A093A602212F43E067EA72E084EA65
:1025700092E00E94C6120E946C03812F0F900F9070
:102580000F90DF91CF911F9108950895FF920F93BF
:102590001F93CF93DF938C01F62ED72FC42F2223C6
:1025A00049F081E080935A020E94E41D9093590201
:1025B0008093580280915A028823C1F0809158027A
:1025C000909159020E94FC1D059780F0EF2DFD2F80
:1025D000D8014C2F50E0CD01801B910B841795073B
:1025E0001CF48D918193F7CF10925A02DF91CF9115
:1025F0001F910F91FF9008950E94E91F0E94E40E21
:102600000C94F51F0E94F91F0E94760F0C94132062
:102610000E94821D0E94D01F0E94D20E0E94FC12B6
:102620000E9402130E94DC0EFBCF8091610280FFAA
:1026300006C06091210170E0660F771F26C081FF00
:1026400004C06091210184E005C082FF07C0609151
:10265000210188E0689FB001112417C090916002A9
:102660009923D1F060912001961788F720912101DC
:1026700088E0289F90011124929FA001939F500D04
:10268000112470E0CA010E9437256038710540F4BA
:102690006115710519F406C068E070E0862F089591
:1026A0008FE7089581E008958091610280FF08C05E
:1026B00060911D0170E0759567957595679521C0CE
:1026C00081FF06C060911D0170E07595679519C086
:1026D00082FF04C060911D0170E010C090915F0204
:1026E000992399F060911C019617A0F780911D0124
:1026F000899FC001112470E00E9437256038710560
:1027000040F46115710519F406C061E070E0862F90
:1027100008958FE7089581E008958D3E21F40E9489
:102720001513819504C08E3E29F40E9415138093E1
:10273000650208958F3E21F40E941513819504C00F
:10274000803F29F40E941513809364020895893F05
:1027500019F40E94541305C08A3F31F40E945413A7
:1027600081958093660208958B3F21F40E94541353
:10277000819504C08C3F29F40E9454138093670212
:1027800008959FE0980F983078F421E030E0A90197
:1027900002C0440F551F9A95E2F7CA019091630257
:1027A000892B8093630208958D3F21F4809161020B
:1027B00081600BC08E3F21F480916102826005C070
:1027C0008F3F29F4809161028460809361020895B3
:1027D0008D3E39F49091650297FF35C010926502E5
:1027E00059C08E3E29F4909165021916BCF32BC096
:1027F000909164028F3E29F497FF25C010926402E5
:1028000049C0803F19F41916CCF31DC0909166029F
:10281000893F29F41916BCF4109266023BC08A3F26
:1028200019F497FF10C0F8CF8B3F39F490916702ED
:1028300097FF09C0109267022DC08C3F21F4909140
:1028400067021916BCF39FE0980F983080F421E0DE
:1028500030E0A90102C0440F551F9A95E2F7CA0162
:1028600080959091630289238093630213C08D3F0A
:1028700021F4809161028E7F0BC08E3F21F4809104
:1028800061028D7F05C08F3F29F4809161028B7FAB
:102890008093610280916402811106C0809165027B
:1028A000811102C01092600280916602811106C0FF
:1028B00080916702811102C010925F0208950E9408
:1028C000E41D20916402211104C02091650222239D
:1028D00021F090935E0280935D02209166022111A7
:1028E00004C020916702222321F090935C02809320
:1028F0005B0282E692E00C94511CEF92FF920F93E0
:102900001F93CF93DF9300D000D000D0CDB7DEB7B8
:1029100086E0E2E6F2E0DE01119601900D928A95E2
:10292000E1F7E0906402F090650200916602109178
:102930006702109264021092650210926602109271
:102940006702E11003C0FF2009F45DC080915D02C1
:1029500090915E020E94FC1DAC019091600299234F
:1029600039F02091220130E02417350758F04BC090
:10297000209123018AE0289F900111242417350714
:1029800018F041C09F3F19F09F5F90936002EE20C6
:1029900061F00E9415131E1414F09FEF01C091E026
:1029A000989F902D112490936402FF2061F00E9463
:1029B00015131F1414F09FEF01C091E0989F902D04
:1029C000112490936502309164023323E1F0209149
:1029D00065022223C1F045EB3403C0011124992381
:1029E00019F09093640203C081E08093640235EB98
:1029F0002303C0011124992319F09093650203C0A9
:102A000081E080936502011103C0112309F45DC0C8
:102A100080915B0290915C020E94FC1DAC01909140
:102A20005F02992339F020911E0130E02417350709
:102A300058F04BC020911F018AE0289F900111247B
:102A40002417350718F041C09F3F19F09F5F9093FE
:102A50005F02002361F00E945413101614F09FEFE0
:102A600001C091E0989F902D11249093660211234C
:102A700061F00E945413111614F09FEF01C091E011
:102A8000989F902D11249093670230916602332312
:102A9000E1F0209167022223C1F045EB3403C0012D
:102AA0001124992319F09093660203C081E080936A
:102AB000660235EB2303C0011124992319F090938A
:102AC000670203C081E080936702809164028111F4
:102AD0000BC080916502811107C08091660281114F
:102AE00003C08091670281110E945F14EB82FC8217
:102AF0000D831E8386E0FE013196A2E6B2E00190CE
:102B00000D928A95E1F726960FB6F894DEBF0FBEB8
:102B1000CDBFDF91CF911F910F91FF90EF9008955E
:102B2000E2E6F2E086E0DF011D928A95E9F7109275
:102B3000600210925F02109261020895EF92FF927C
:102B40000F931F93CF93DF938B01682F11110AC04E
:102B5000442329F0E82FF0E0E051FF4F6491762FF5
:102B6000862F75C0212F30E0E82FF0E0442321F0BC
:102B7000E051FF4FE491F0E046E0049FC0011124D2
:102B8000CFEFD0E0BE010E9423254BEA4603C001EF
:102B9000479F900D1124800F911D800F911D982F3C
:102BA000990F890FAE01421B530B4E9FD0014F9FCF
:102BB000B00D5E9FB00D11249B2F189FA001112412
:102BC000452F55278E01041B150B0E9FA0010F9F4B
:102BD000500D1E9F500D11247E01E81AF108E29E4F
:102BE0008001E39E100DF29E100D1124212F33273A
:102BF000C21BD30BCE9F9001CF9F300DDE9F300DB7
:102C0000112462307105A9F048F46115710569F06D
:102C100061307105C9F48B2F752F0DC064307105BB
:102C200081F058F06630710579F47E2F8B2F932F49
:102C30000DC0832F7B2F9E2F09C08E2F7B2F952FAA
:102C400005C08E2F732F02C07E2F852F692FDF9135
:102C5000CF911F910F91FF90EF90089541E00E9456
:102C60009E1508950E942E160895CF93DF93762F18
:102C7000E901682F842F0E943216798368838A8342
:102C8000DF91CF910895413F08F040EF0C94351645
:102C90008091AA02982F9695913021F081708260E0
:102CA0008093AA028091AD02813F18F080EF80935B
:102CB000AD02089588E090E00C946625CF92DF92F3
:102CC000EF92FF926B017C010E944816B701A601AA
:102CD00088E090E0FF90EF90DF90CF900C948425F7
:102CE000EAEAF2E083E0808311828FEF828380EF53
:102CF0008383148260817181828193810C945E163A
:102D00009091AE02933018F49F5F9093AE028823A7
:102D100051F06091AA027091AB028091AC02909147
:102D2000AD020C945E16089581E00C94801690918B
:102D3000AE02992319F091509093AE02882351F07E
:102D40006091AA027091AB028091AC029091AD02A9
:102D50000C945E16089581E00C94971670E00C9424
:102D6000BF18609125018091AA0280FF0AC080915E
:102D7000240123E0829FC001112481559D4F0C94B2
:102D8000AE168091260190912701891780F7E82FD0
:102D9000F0E09F01220F331FE20FF31FE155FD4FBB
:102DA0001182108212828F5FF0CFEAEAF2E0808116
:102DB0008E7F808360817181828193810E945E1603
:102DC0002FEF80E792E0215080409040E1F700C073
:102DD00000000C94B116EAEAF2E080818E7F8083D5
:102DE0002FEF80E792E0215080409040E1F700C053
:102DF00000000C94B1169091AA0290FF16C0909119
:102E0000260120912701921770F4E92FF0E0DF01ED
:102E1000AA0FBB1FEA0FFB1FE155FD4F81836083A3
:102E200042839F5FF0CF0C94B1160895EF92FF920A
:102E30000F931F93CF93DF9300D01F92CDB7DEB7D0
:102E40009091AA0290FF2CC0E22E142F062FF82E8C
:102E5000E92FE695F0E0E156FE4F8081809369020C
:102E60009E7F923059F49E012F5F3F4F8F2D0E941D
:102E700043164B8169818A810E94FB16F092AB0256
:102E80000093AC021093AD02EE2051F06091AA02C3
:102E90007091AB028091AC029091AD020E945E16DF
:102EA0000F900F900F90DF91CF911F910F91FF9096
:102EB000EF900895EAEAF2E09181282F4381628140
:102EC00088E0890F0C94161781E00C945A17EAEAEF
:102ED000F2E09181282F4381628188EF890F0C9461
:102EE000161781E00C946717EAEAF2E0628128E0A5
:102EF000620F08F46FEF282F438181810C9416171D
:102F000081E00C947417EAEAF2E0628128E0621B27
:102F100008F460E0282F438181810C94161781E02A
:102F20000C948317EAEAF2E0438128E0420F08F4A8
:102F30004FEF282F628181810C94161780E00C944A
:102F4000921781E00C949217EAEAF2E0438128E0BC
:102F5000421B08F440E0282F628181810C941617EF
:102F600080E00C94A41781E00C94A41720E00C944A
:102F700016178091AA0280FF18C08170826080932A
:102F8000AA02662351F06091AA027091AB0280916F
:102F9000AC029091AD020E945E164091AD0260912C
:102FA000AC028091AB020C94B6170895682F81E0B3
:102FB0000C94B91780E00C94D61781E00C94D617C6
:102FC000682F9091AA0296958FEF890F09F481E0FE
:102FD0000C94B91781E00C94E01761E00C94B917D8
:102FE000EAEAF2E080818160808386950C94ED1797
:102FF0008091AA0280FD0C94D5160C94F01760E025
:103000000C94B9178091680281112CC00E94E70DC1
:10301000811104C00E948F0E0E9470160E945A16E1
:103020006093AA027093AB028093AC029093AD02BE
:103030006E7F61F40E9470160E945A166093AA0275
:103040007093AB028093AC029093AD020E9448163D
:103050008091AA0280FF03C086950E94FF1781E03D
:10306000809368020895EAEAF2E0808181608083BB
:1030700086950C94FF178091AA0280FD0C94EB16A4
:103080000C943318882311F0FA0101C0FB01099454
:103090001F93CF93DF93FB01128111116BC0EC01E1
:1030A0000E94FE0C8272CA3CFCE5DF0709F450C0A6
:1030B000C0F4C63CECE5DE07E1F148F4C43C9CE515
:1030C000D90759F178F5C33CDC4521F121C0C83C52
:1030D0009CE5D90799F1B8F544E657E161E777E156
:1030E00025C0CE3CFCE5DF0709F441C050F4CC3CE0
:1030F000ECE5DE0791F1B0F541EA57E163EB77E1EA
:1031000015C0C73D8CE5D807A8F1CE35DD4591F156
:1031100011E030C00E94F8172DC04AEE57E16DED66
:1031200077E104C04DED57E16AEE77E10E94421865
:1031300021C041E757E164E677E1F8CF4FE857E176
:1031400060E877E1F3CF40E857E16FE877E1EECF51
:1031500043EB57E161EA77E1E9CF4BEA56E164E9F5
:1031600076E1E4CF44E956E16BEA76E1DFCF81E036
:103170000E94ED17812FDF91CF911F910895539AEF
:103180002BB1277F3BB138604FB7F894FC01CB01DE
:10319000880F991F680F791F6E0F7F1FE617F707BB
:1031A00089F0819198E03BB9000000C087FF2BB9FE
:1031B000880F000000C000C000C02BB900C09A9565
:1031C00091F7ECCF4FBF8FE594E00197F1F700C086
:1031D00000000895CF93DF93EC01FB0182818823E7
:1031E00009F43CC1C430FDE5DF0760F4CB3F9CE54A
:1031F000D90788F49E0122503C452431310508F05E
:103200002EC109C0C236EDE5DE0729F0C63AFDE55C
:10321000DF0709F024C10E94FA0D9093A302809366
:10322000A202C1318CE5D80709F4C6C008F042C03B
:10323000C930ECE5DE0709F49BC000F5C5308CE52C
:10324000D80709F485C078F4C330ECE5DE0709F44B
:1032500078C008F07AC0C230DC4509F0F5C0809132
:10326000A2028160EFC0C7309CE5D90709F478C09D
:1032700008F07AC08091A2028061E4C0CD30FCE504
:10328000DF0709F487C058F4CB309CE5D90709F46F
:1032900079C008F07BC08091A20288606FC0CF30F7
:1032A000FCE5DF0709F480C008F082C08091A2022B
:1032B000877FC8C0CE3F9CE5D90709F471C000F5EF
:1032C000C531FCE5DF0709F485C068F4C3319CE52E
:1032D000D90709F475C008F095C00E94AD07809128
:1032E000A2028F77AFC0CC3FFCE5DF07A9F108F061
:1032F00054C0CB3FDC4509F0A7C08091A30240C079
:10330000C230EDE5DE0709F489C058F4C1158DE53A
:10331000D80709F45AC008F069C08091A3028260FE
:103320002FC0C236EDE5DE0709F47CC0C63AFDE5E4
:10333000DF0709F481C0C330DD4509F085C080E0B6
:103340006EC08091A20282607DC08091A20216C0F0
:103350008091A202886076C08091A30282604FC0F3
:103360008091A20280626EC08091A20280646AC0D5
:103370000E94AD078091A202806864C0846062C030
:1033800081603DC08091A2028E7F5CC08091A202CC
:103390008D7F58C08091A20216C08091A30218C0F0
:1033A0008091A3028D7F2BC08091A2028F7E4AC0A4
:1033B0008091A2028F7D46C08091A2028F7B42C085
:1033C0008091A202877F8B7F3DC08091A3028D7F79
:1033D0008E7F15C08091A20282FB222720F991E006
:1033E000922790FB82F990FB83F92CC08091A30275
:1033F000982F909591708E7F892B90FB81F9809307
:10340000A30222C00E94AD078091A20287FB22275F
:1034100020F991E0922790FB87F914C081E00E9487
:10342000910E12C08091A20284FB222720F991E024
:10343000922790FB84F906C08091A202982F909564
:1034400090FB80F98093A2028091A2029091A30246
:103450000E940B0E0E94AD0780E001C081E0DF9169
:10346000CF9108958FE891E00197F1F700C0000037
:1034700008950C943C02CF93DF93A3EBB1E0C1EB32
:10348000D1E021E030E071E0A53BB70759F18D9123
:10349000E82FE295EF70F0E041A18F70B90102C012
:1034A000660F771F8A95E2F7CB01962F90959423AC
:1034B00091A392A1892B82A38991E82FE295EF70C5
:1034C000F0E041A18F70B90102C0660F771F8A95A5
:1034D000E2F7CB01962F9095942391A392A1892B8B
:1034E00082A3D1CF0E94321A89B1982F9170499945
:1034F00002C080E001C082E0892B80936F0283B11B
:1035000085FB882780F94E9902C090E001C092E0C7
:10351000892B80937002DF91CF9108954F925F9233
:103520006F927F928F929F92AF92BF92CF92DF92D3
:10353000EF92FF920F931F93CF93DF930FE612E06A
:1035400083EBC82E81E0D82E91EBE92E91E0F92E85
:103550002DE6822E22E0922ECBE6D2E05801512CAD
:10356000412C34E0632E712CD501ED915D014E2F7D
:10357000440F440FF60121916F01E22FE295EF70A5
:10358000F0E080A190E02F7002C0959587952A9574
:10359000E2F781709927D7015D917D01E52FE295D2
:1035A000EF70F0E020A130E05F7002C03595279504
:1035B0005A95E2F7F901E170FF2720FF02C0E2E02F
:1035C000F0E0E82BF92BE42BD801ED938D01EF709F
:1035D000F0E0EF55FE4F9081F4018081890F8083E8
:1035E00084304CF088818F5F888360E0852D0E9455
:1035F000391A21E001C020E0D4018C918D3F44F4C0
:1036000088818150888361E0852D0E94391A21E0EC
:10361000F4018081082E000C990BB3010E9437251C
:10362000D4018D934D01422A53942196B2E05B124E
:103630009BCF842DDF91CF911F910F91FF90EF9041
:10364000DF90CF90BF90AF909F908F907F906F90C2
:103650005F904F900895CF93DF9386319C4541F55D
:10366000EB010E94FE0C982F8A8120911A01309163
:103670001B01882379F09A7A81E009F480E0809335
:103680007102911102C069E201C065E3C9010E94A3
:10369000211D0AC080917102811102C069E201C03E
:1036A00065E3C9010E942C1D0E94400D80E001C00D
:1036B00081E0DF91CF9108950F931F93CF93DF9314
:1036C000C42FD22FFC0182818823C9F04093740259
:1036D0000E94E41D909373028093720280E28C0F2B
:1036E000883008F057C0C77081E001C0880FCA95C4
:1036F000EAF7DF91CF911F910F910C94FC04809118
:103700007402481330C080917202909173020E943B
:10371000FC1D883C910538F510E21D0FCD17B9F05E
:1037200080E28C0F883040F4C77081E001C0880FC0
:10373000CA95EAF70E940305183028F581E09D2F0D
:10374000977001C0880F9A95EAF70E94FC04802FB9
:103750000E94F3041830F0F4D77081E001C0880FA4
:10376000DA95EAF70AC080E28C0F883098F4C770C7
:1037700081E001C0880FCA95EAF7DF91CF911F91D0
:103780000F910C940305802FDF91CF911F910F9122
:103790000C94F304DF91CF911F910F9108950F9333
:1037A0009C01CB01243F4CE5340731F188F4293DDD
:1037B000FCE53F07D9F02A3D4CE5340779F1283D77
:1037C0003C45A9F506E221EE41EE68ED7CE52BC013
:1037D000263FFCE53F07E1F0A8F0273F3C4539F5DF
:1037E00007E225EE46EE67EF7CE51DC007E225EE19
:1037F00045EE69ED7CE517C006E221EE40EE64EF90
:103800007CE511C007E225EE44EE65EF7CE50BC0D8
:1038100006E221EE42EE66EF7CE505C008E221E01B
:1038200045EE6AED7CE50E945C1B80E008C0FC016F
:103830008281882319F01092740201C081E00F91F7
:1038400008959093B7018093B601089590937A02FA
:10385000809379020895E0917902F0917A0230978D
:1038600021F00190F081E02D099480E00895E0912D
:103870007902F0917A02309799F020913501222354
:1038800059F02091A20227FF07C0DC012C9111966C
:103890002C93119726E02C930280F381E02D09945C
:1038A0000895E0917902F0917A02309739F022E0A0
:1038B000DC012C930480F581E02D0994089520917A
:1038C0007702309178022817390771F090937802C7
:1038D00080937702E0917902F0917A02309721F09B
:1038E0000680F781E02D09940895209175023091AA
:1038F00076022817390771F090937602809375024B
:10390000E0917902F0917A02309721F00084F185FC
:10391000E02D09940895FC013296809135018823A9
:1039200031F08091A20287FF02C09EE101C096E0C3
:1039300080E0915028F021912223D9F38F5FF9CFB5
:103940000895662351F1209135012223E9F0209159
:10395000A20227FF19C0462F4695469546954E313F
:10396000E0F4677021E030E002C0220F331F6A9557
:10397000E2F7FC01E40FF11D828190E02823392356
:1039800081E0232B69F409C0FC013296089621914D
:10399000621729F0E817F907D1F780E0089581E070
:1039A00008959C01FC0132969FEF80E041914617FB
:1039B00089F09F3F19F4411101C0982F8F5F863025
:1039C000A9F79F3F39F0F901E90FF11D97FDFA952D
:1039D0006283089508959C012A5F3F4FFC01428154
:1039E000461301C01282019682179307B9F7089512
:1039F000262F2695269526952E3168F4FC01E20F98
:103A0000F11D677021E030E001C0220F6A95EAF7EE
:103A10008281282B22830895262F26952695269588
:103A20002E3170F4FC01E20FF11D677021E030E0EF
:103A300001C0220F6A95EAF720958281282322830C
:103A4000089520913501222329F02091A20227FD1B
:103A50000C94F81C0C94D11C20913501222329F0E0
:103A60002091A20227FD0C940C1D0C94EB1C2091BC
:103A70003501FC013296222331F08091A20287FFAA
:103A800002C08EE101C086E0DF011D928A95E9F750
:103A9000089508950C94491D83E080937B020C9453
:103AA0004A1D811102C081E001C082E080937B0247
:103AB0000C944A1D0C94511D81E080937B020C9460
:103AC0004A1D0C945C1D08950C94631D0C94641D98
:103AD0000C94631D0C94631D0C94631DCF930E9482
:103AE0006A1D0E9482120E94681DC0E08C2F0E94F5
:103AF000C511811104C0CF5FC330C1F701C081E09F
:103B0000CF91089508951F920F920FB60F9211242E
:103B10008F939F93AF93BF9380917C02811113C0C9
:103B20008091BB029091BC02A091BD02B091BE02F7
:103B30004196A11DB11D8093BB029093BC02A0933E
:103B4000BD02B093BE02BF91AF919F918F910F9034
:103B50000FBE0F901F9018958091C302843031F1F1
:103B60000E94D70310927C0220E488E190E00FB617
:103B7000F894A895809360000FBE2093600083B7EF
:103B8000817F846083BF83B7816083BF7894889589
:103B900083B78E7F83BF0FB6F894A895809160009D
:103BA000886180936000109260000FBE08950E94AB
:103BB000AD070C94DB0382E084BD93E095BD9AEFE2
:103BC00097BD80936E0008952FB7F8948091BB0243
:103BD0009091BC02A091BD02B091BE022FBF08958A
:103BE0002FB7F8946091BB027091BC028091BD0226
:103BF0009091BE022FBF08959C014FB7F894809119
:103C0000BB029091BC02A091BD02B091BE024FBF19
:103C1000821B930B089578941F920F920FB60F9208
:103C200011248F939F93AF93BF938091BB02909188
:103C3000BC02A091BD02B091BE020196A11DB11DB2
:103C40008093BB029093BC02A093BD02B093BE02CE
:103C5000BF91AF919F918F910F900FBE0F901F90CA
:103C6000189587E797E790930108809300089AE0FA
:103C700088E10FB6F894A895809360000FBE9093EA
:103C80006000FFCF8091A0020895089522E0209364
:103C9000E9002FEF3091E800215035FD06C035EDE9
:103CA0003A95F1F700002111F5CF2091E80025FFAA
:103CB0000BC040E050E066E070E00E9485208091FB
:103CC000E8008E778093E8000895CF93DF932091EA
:103CD0003501222339F02091A20227FF03C060E2C0
:103CE00022E002C068E021E02093E9002FEF30914C
:103CF000E800215035FD06C035ED3A95F1F700009A
:103D00002111F5CF2091E80025FF1DC0EC01809125
:103D10003501811105C040E050E068E070E003C06B
:103D200070E040E050E0CE010E9485208091E800E4
:103D30008E778093E80080E2FE01A0E8B2E0019077
:103D40000D928A95E1F7DF91CF91089580937D02DE
:103D500070937F0260937E028091C302843001F5EC
:103D600082E08093E9008FEF9091E800815095FD0B
:103D700006C095ED9A95F1F700008111F5CF80917D
:103D8000E80085FF0DC040E050E063E070E08DE7A3
:103D900092E00E9485208091E8008E778093E80071
:103DA0000895BC0184E00C94A61EBC0183E00C9431
:103DB000A61E8091C202811109C00E9416220E9493
:103DC00073228091E20084608093E2000895109253
:103DD000C20208950C94611D6091BF0281E06111DF
:103DE00001C080E00C944C1D9091C30281E094309E
:103DF00009F080E06091BF020C94511D42E061EC3B
:103E000081E00E948F2142E261EC82E00E948F21DA
:103E10009091C30281E0943009F080E06091BF028C
:103E20000C945A1D8091C502833009F461C030F4AE
:103E3000813071F0823009F49AC008958A3009F413
:103E400086C08B3009F46CC0893009F0A8C020C04E
:103E50008091C402813A09F0A2C08091E800877F76
:103E60008093E8008091C8029091C902892B21F4C7
:103E700060E280E892E003C060E080E090E070E003
:103E80000E94D0208091E8008B778093E80008950D
:103E90008091C402813209F082C08091C802909161
:103EA000C902029708F07BC08091E800877F809369
:103EB000E8008091E80082FD05C08091C302811175
:103EC000F8CF6DC02091F3008091F20090E0922B2A
:103ED000029731F48091F100813011F0863021F4A5
:103EE0008091F1008093A0028091E8008B7753C00D
:103EF0008091C402813A09F052C08091C802909129
:103F0000C902892B09F04BC08091E800877F80931C
:103F1000E8008091E80080FFFCCF8091350136C039
:103F20008091C4028132D9F58091C8029091C90272
:103F3000892BA9F58091E800877F8093E8000E9493
:103F4000C4218091C602809335010C94AD07809105
:103F5000C402813221F58091E800877F8093E800D8
:103F60000E94C4218091C7028093A102089580918C
:103F7000C402813AA1F48091E800877F8093E80031
:103F80008091E80080FFFCCF8091A1028093F10036
:103F90008091E8008E778093E8000C94C421089506
:103FA00084B7877F84BF0FB6F894A895809160008E
:103FB000886180936000109260000FBE90E080E8FE
:103FC0000FB6F89480936100909361000FBE0C943B
:103FD0005C1D0E9416220E947322E2EEF0E08081B6
:103FE0008460808378940C94082589E291E00C9495
:103FF000261C8091C3028530A9F48091C3028530CC
:1040000079F40E94AC1D8091C1028823B1F30E9413
:104010006E1D882391F30E946F200E94AD07EDCFA3
:104020000C94D71D089508950C941620292F33273A
:1040300023303105C9F060F42130310581F02230A0
:10404000310509F044C08BE390E022E132E043C047
:1040500021323105E1F02232310549F138C082E1E7
:1040600090E02DE432E037C099278130910549F086
:1040700028F0029761F5E0EFF1E005C0EEE0F2E034
:1040800002C0E2E0F2E0849190E09F0124C061155B
:10409000710541F061307105D1F489E090E02DE3C4
:1040A00032E019C089E090E024E232E014C06115EA
:1040B000710541F06130710551F486EB90E02FE518
:1040C00032E009C080E490E025E133E004C080E004
:1040D00090E020E030E0FA0131832083089580E110
:1040E00089BD82E189BD09B400FEFDCF8091D80071
:1040F0008F7D8093D8008091E00082608093E00003
:104100008091E00081FDFCCF0895CF92DF92EF9285
:10411000FF920F931F93CF93DF93EC018B017A01F2
:104120000E94E321811133C0E114F10439F0F70159
:1041300080819181081B190BC80FD91FC12CD12C6C
:104140000115110519F18091E80085FD16C08091D7
:10415000E8008E778093E800E114F10449F0F7015C
:1041600080819181C80ED91ED182C08285E00FC0A6
:104170000E94E321882321F30AC089918093F100F2
:1041800001501109FFEFCF1ADF0ADACF80E0DF918B
:10419000CF911F910F91FF90EF90DF90CF900895F6
:1041A0002091CA023091CB022617370748F06115DB
:1041B000710539F42091E8002E772093E80001C0C2
:1041C000B901FC0120E06115710579F18091C3020C
:1041D0008823F1F18530F1F18091E80083FD3CC046
:1041E0008091E80082FD2EC08091E80080FFEBCF37
:1041F0002091F3008091F20090E0922B61157105FF
:1042000051F08830910538F421912093F1006150EC
:1042100071090196F3CF21E0089709F020E0809121
:10422000E8008E778093E800CECF2111CFCF0AC06F
:104230008091C302882361F0853061F08091E800AD
:1042400083FD0AC08091E80082FFF2CF80E00895EC
:1042500082E0089583E0089581E008952091CA02E4
:104260003091CB022617370748F06115710539F4F4
:104270002091E8002E772093E80001C0B901FC01ED
:1042800020E06115710591F18091C302882309F442
:1042900040C0853009F43FC08091E80083FD3DC0F7
:1042A0008091E80082FD2FC08091E80080FFE9CF77
:1042B0002091F3008091F20090E0922B611571053E
:1042C00059F08830910540F424912093F100319603
:1042D000615071090196F2CF21E0089709F020E0C2
:1042E0008091E8008E778093E800CBCF2111CCCF6E
:1042F0000AC08091C302882361F0853061F080910B
:10430000E80083FD0AC08091E80082FFF2CF80E0E0
:10431000089582E0089583E0089581E00895982F3C
:10432000973068F59093E900981739F07091EC0098
:104330002091ED005091F00003C0242F762F50E023
:1043400021FD02C09F5FECCF3091EB003E7F3093A8
:10435000EB003091ED003D7F3093ED003091EB00AC
:1043600031603093EB007093EC002093ED0050939C
:10437000F0002091EE0027FDE5CF80E008958F70DA
:104380008093E90081E008958091C40287FF11C005
:104390008091E80082FD05C08091C3028111F8CFB1
:1043A00011C08091E8008B770BC08091C3028823F5
:1043B00049F08091E80080FFF8CF8091E8008E7787
:1043C0008093E80008952091E4003091E50095E69F
:1043D0004091EC00842F817040FF23C08091E80061
:1043E00080FD1DC08091C302882399F0853099F02B
:1043F0008091EB0085FD11C04091E4005091E500F3
:104400002417350729F3915011F09A01E1CF84E088
:10441000089582E0089583E0089581E0089580E0A2
:1044200008954091E80042FFDDCF08950E94842264
:104430000E948C22E0EEF0E0808181608083E8EDD4
:10444000F0E080818F77808319BCA7EDB0E08C917C
:104450008E7F8C9380818F7E80831092C20208951C
:104460000F931F93CF93DF930E9484220E948C228C
:10447000C8EDD0E088818F778883888180688883C1
:1044800088818F7D888319BC1092C3021092BF026D
:104490001092C1021092C00200EE10E0F80180817B
:1044A0008B7F808388818160888342E060E080E048
:1044B0000E948F21E1EEF0E080818E7F8083E2EE2A
:1044C000F0E0808181608083808188608083F80152
:1044D00080818E7F8083888180618883DF91CF9106
:1044E0001F910F910895E8EDF0E080818F7E808329
:1044F000E7EDF0E080818160808384E082BF81E02D
:104500008093C2020C943022E8EDF0E080818E7F2F
:1045100080831092E20008951092DA001092E10078
:1045200008951F920F920FB60F9211242F933F936D
:104530004F935F936F937F938F939F93AF93BF93AB
:10454000EF93FF938091E10082FF0BC08091E20026
:1045500082FF07C08091E1008B7F8093E1000E9481
:1045600007258091DA0080FF1FC08091D80080FF6E
:104570001BC08091DA008E7F8093DA008091D90091
:1045800080FF0DC080E189BD82E189BD09B400FED4
:10459000FDCF81E08093C3020E94D91E05C019BCE3
:1045A0001092C3020E94E71E8091E10080FF19C0B3
:1045B0008091E20080FF15C08091E2008E7F8093A1
:1045C000E2008091E20080618093E2008091D80057
:1045D00080628093D80019BC85E08093C3020E945A
:1045E000EC1E8091E10084FF30C08091E20084FFE6
:1045F0002CC080E189BD82E189BD09B400FEFDCFF8
:104600008091D8008F7D8093D8008091E1008F7ECB
:104610008093E1008091E2008F7E8093E2008091A0
:10462000E20081608093E2008091BF02882311F054
:1046300084E007C08091E30087FD02C081E001C0F3
:1046400083E08093C3020E94F41E8091E10083FF07
:1046500029C08091E20083FF25C08091E100877F1F
:104660008093E10082E08093C3021092BF028091A8
:10467000E1008E7F8093E1008091E2008E7F809345
:10468000E2008091E20080618093E20042E060E01D
:1046900080E00E948F218091F00088608093F0007C
:1046A0000E94EA1EFF91EF91BF91AF919F918F9170
:1046B0007F916F915F914F913F912F910F900FBE1E
:1046C0000F901F9018951F920F920FB60F92112402
:1046D0002F933F934F935F936F937F938F939F930A
:1046E000AF93BF93CF93DF93EF93FF93C091E90014
:1046F000CF708091EC00D82FD17080FDD0E810925F
:10470000E9008091F000877F8093F00078940E9408
:10471000A7231092E9008091F00088608093F00058
:10472000CD2BCF70C093E900FF91EF91DF91CF9136
:10473000BF91AF919F918F917F916F915F914F91B9
:104740003F912F910F900FBE0F901F9018951F93C0
:10475000CF93DF93CDB7DEB7AA970FB6F894DEBF3D
:104760000FBECDBFE4ECF2E08091F100819322E036
:10477000EC3CF207C9F70E94121F8091E80083FF0A
:104780002EC18091C4029091C502492F50E04A3059
:10479000510508F024C1FA01EE59FF4F0C944B2546
:1047A000803821F0823809F01AC108C08091C00217
:1047B0009091C102992389F082600FC08091C80254
:1047C0008F70873008F00BC18093E9008091EB0077
:1047D00085FB882780F91092E9009091E800977F87
:1047E0009093E8008093F1001092F100D1C0282F3F
:1047F0002D7F09F0F4C0882319F0823061F0EFC0FA
:104800008091C602813009F0EAC0933009F080E05F
:104810008093C1022EC08091C60281112AC080916E
:10482000C8028F702FEF280F263008F0D8C0809371
:10483000E9002091EB0020FF1CC0933021F480910F
:10484000EB00806214C09091EB0090619093EB00BC
:1048500021E030E0A90102C0440F551F8A95E2F71C
:104860004093EA001092EA008091EB008860809308
:10487000EB001092E9008091E800877F8093E800C8
:104880000E94C421ACC08111AAC01091C6021F773A
:104890008091E3008078812B8093E3008091E80091
:1048A000877F8093E8000E94C4218091E80080FF08
:1048B000FCCF8091E30080688093E300111102C077
:1048C00082E001C083E08093C30289C080588230B7
:1048D00008F085C08091C6029091C7028C3D53E0DC
:1048E000950779F583E08A838AE289834FB7F89444
:1048F000DE01139620E03EE051E2E32FF0E050931A
:104900005700E49120FF03C0E295EF703F5FEF7026
:104910008E2F90E0EA3010F0C79601C0C0968D93BC
:104920009D932F5F243149F74FBF8091E800877F27
:104930008093E8006AE270E0CE0101960E94D020E8
:1049400016C06091C8027091C902AE014F5F5F4FFF
:104950000E941420BC01892B09F441C09091E80009
:10496000977F9093E80089819A810E942E218091FF
:10497000E8008B778093E80032C0803881F5809121
:10498000E800877F8093E8008091BF028093F10068
:104990008091E8008E7772CF811121C08091C6028C
:1049A0009091C70299270297D4F48091E800877FFD
:1049B0008093E8008091C6028093BF020E94C421C8
:1049C0008091BF02811106C08091E30087FD02C083
:1049D00081E001C084E08093C3020E94FE1E8091AA
:1049E000E80083FF0AC08091E800877F8093E80099
:1049F0008091EB0080628093EB00AA960FB6F8944A
:104A0000DEBF0FBECDBFDF91CF911F9108950895F6
:104A1000CF938091C3028823A1F0C091E900CF70A9
:104A20009091EC00892F817090FD80E8C82B109246
:104A3000E9008091E80083FD0E94A723CF70C09316
:104A4000E900CF910895AA1BBB1B51E107C0AA1F23
:104A5000BB1FA617B70710F0A61BB70B881F991F1F
:104A60005A95A9F780959095BC01CD01089597FBC3
:104A7000072E16F4009407D077FD09D00E94232555
:104A800007FC05D03EF4909581959F4F0895709551
:104A900061957F4F0895EE0FFF1F0590F491E02D73
:104AA0000994FB01DC0104C08D910190801921F46F
:104AB00041505040C8F7881B990B0895F999FECFD3
:104AC00092BD81BDF89A992780B50895A6E1B0E01E
:104AD00044E050E00C949825A8E1B0E042E050E0BA
:104AE0000C949825262FF999FECF92BD81BDF89A96
:104AF000019700B4021639F01FBA20BD0FB6F89422
:104B0000FA9AF99A0FBE08950396272F0E947325EB
:104B10000E947225252F0E947325242F0C94732543
:104B20000196272F0E9473250C947225DC01CB017E
:104B3000FC01F999FECF06C0F2BDE1BDF89A3196AD
:104B400000B40D9241505040B8F70895F894FFCF4B
:104B5000010001000100010001000100010001004D
:104B60000100010001000100C800260228085001D0
:104B70001E0A14010004000404421E651E461ED5D0
:104B80001ED11E451E01E200E900EA00B500B60094
:104B9000B700CD008301CC008A019201940121026B
:104BA000230224022502260227022A02B300B400AF
:104BB0006F007000818283E200E900EA00B500B670
:104BC00000B700CD008301CC008A0192019401213D
:104BD00002230224022502260227022A02B300B47D
:104BE000006F007000818283F0F1F4F567F7F60042
:104BF0000100FF0100010000FFFF0000010001FFB4
:064C0000009196903500C2
:00000001FF
